:020000020000FC
:1000000012C06DC36DC36DC36DC36DC36DC36DC3CE
:100010006DC36DC391C391C391C391C391C3EFC32A
:10002000EFC3F0C3F0C304E00EBF0FE50DBF78943B
:100030000FEF01BB03EC07BB0CE304BB08BB0027BD
:1000400002BB05BBF6D222243324442404E6502EFE
:1000500000936D0000936E0000936F00009370009A
:1000600003E003BF01E009BFF894002702BF0DBD04
:100070000CBD0EE806B900E110E00ABD1BBDAAD315
:10008000789475D204D052D1E8D031D1FACFB29B56
:100090000DC0B49B05C0B59B1FC0B39B79C008952C
:1000A00008E0302E02E000937000089560D2B29B09
:1000B000FDCF03E000937000032D18E0312E0030D7
:1000C00051F000916600033631F00395009366000D
:1000D00010E1A4D2F9D2089506E0302E48D2032DC3
:1000E0000030E9F0B59BFACF00916900003059F07B
:1000F00000917400003041F000270093740011E17A
:100100008DD2AC98E1D2089501E00093740011E122
:1001100085D2AC9AAD9804E6502ED6D20895B39B02
:1001200091C000917000003019F00130C9F00895BD
:1001300001E0009369001AE071D200916000009321
:1001400067001CE06BD200916100009368001BE027
:1001500065D2BDD20CD2EAD0B59BFCCFB5D2089502
:1001600002E0009369001AE059D200916200009306
:1001700067001CE053D200916300009368001BE00D
:100180004DD2A5D2F4D1D2D0B59BFCCF9DD208954B
:1001900006E0302EECD1032D0030E9F0B39BFACF0E
:1001A00000916C00003059F000917400003041F073
:1001B00000270093740011E131D2AD9885D20895E3
:1001C00002E00093740011E129D2AD9AAC9804E6E4
:1001D000502E7AD2089500917000003019F001304D
:1001E000C9F0089501E000936C001DE017D2009162
:1001F000600000936A001FE011D20091610000933B
:100200006B001EE00BD263D291D0B1D1B39BFCCF77
:100210005BD2089502E000936C001DE0FFD10091D5
:10022000620000936A001FE0F9D10091630000931F
:100230006B001EE0F3D14BD279D099D1B39BFCCFA8
:1002400043D208951FD2F5D142D244D240D242D2F5
:1002500038D240D236D23ED214CF032D003099F49A
:1002600000917100023641F5009162001091630027
:10027000889400581C4020F001E00093700003C0F7
:10028000002700937000009171000236A9F40091DC
:100290007000033029F4112700916600C4D008953E
:1002A00000917000023049F40091640010916500E3
:1002B00058D1B9D08FD208950895009170000130BF
:1002C00059F000916000109161004BD1ACD082D206
:1002D0000027009370000895009162001091630060
:1002E00040D1A1D077D201E0009370000895009131
:1002F0007400023091F0013099F0009169000030F3
:1003000021F000917300013059F000916C00003031
:1003100051F000917300013031F0AA98AB9A089522
:10032000AA9AAB980895AA98AB9808950091710085
:100330000236B9F5052D0030A1F5009174000030AA
:1003400081F1033071F140917400013061F000914E
:100350006A0010916B0020916C0030917000339511
:100360003217F9F40BC000916700109168002091DA
:100370006900309170003395321799F42091700024
:10038000213029F0209160003091610004C020915B
:1003900062003091630040917400413019F04230A6
:1003A00031F0089588940217130730F00895889467
:1003B0002017310790F0089500916600003009F190
:1003C0000130F9F0AC98AD9A04E6502E02E00093AB
:1003D000740011E123D17BD10895009166000030B3
:1003E00081F0AD98AC9A0A950093660010E116D1A1
:1003F00004E6502E01E00093740011E10FD167D1A3
:10040000089503E00093740011E108D100270093E0
:10041000660010E103D1AC98AD9863E058D15AD191
:100420006A95E1F7089522270456120B50F10456FD
:10043000120BA8F10456120BB0F10456120BB8F1CE
:100440000456120BC0F10456120BC8F10456120BDD
:10045000D0F10456120BD8F10456120BE0F10456F9
:10046000120BE8F140917000403059F0423049F0F1
:100470004AE040936F004BE040936E0040936D0064
:10048000089530917000303031F0323021F04CE07E
:1004900040936F0027C0442740936F0023C041E082
:1004A00040936F001FC042E040936F001BC043E0C9
:1004B00040936F0017C044E040936F0013C045E0C5
:1004C00040936F000FC046E040936F000BC047E0C1
:1004D00040936F0007C048E040936F0003C049E0BD
:1004E00040936F000C590A50A8F00A50B8F00A5017
:1004F000C8F00A50D8F00A50E8F00A50F8F00A5054
:1005000008F10A5018F10A5028F10A5049E04093C6
:100510006E0023C040E040936E001FC041E0409356
:100520006E001BC042E040936E0017C043E0409352
:100530006E0013C044E040936E000FC045E040934E
:100540006E000BC046E040936E0007C047E040934A
:100550006E0003C048E040936E00065F00936D009C
:10056000089525E0169507952A95E1F708950091DD
:100570007400033021F400917300013039F11091BF
:100580006D00C798C69AC09A27D012BB34D010917C
:100590006E00C698C79AC09A1FD012BB0091700017
:1005A000013009F4929A27D0929810916F00C09868
:1005B000C69AC79A11D012BB00917000013019F091
:1005C000033009F0929A17D092980895002702BB41
:1005D000C098C698C7980895E8EEF5E020E0E10FCE
:1005E000F21FC895102D0895FA42D9CB63ABBBC258
:1005F000FBEBB91100011F932F9312E328E21A9528
:10060000F1F72A95E1F72F911F910895E199FECF17
:1006100022271EBB2FBBE09A0DB30895E199FECFB0
:10062000F89422271EBB2FBB0DBBE29AE19A789467
:1006300008951AE0EBDF009369001BE0E7DF009309
:1006400068001CE0E3DF009367001DE0DFDF00933C
:100650006C001EE0DBDF00936B001FE0D7DF009330
:100660006A0010E1D3DF0093660011E1CFDF009351
:100670007400013019F0023019F00895AC9A089511
:10068000AD9A089538E01AE00027C8DF13953A952F
:10069000D9F70895042D003079F00FB5003009F036
:1006A0000895F89400E40FBD09E00EBD04E10BBD10
:1006B00005E30ABD7894089500270FBD0EBDC198CB
:1006C000089504E1402E089503E2402E089504E6C3
:1006D000402E089554E64BDF5A95E9F70895189592
:1006E00018951895189518951895189518950F93AD
:1006F0009FB7D0DF2394022D003079F4009173006E
:10070000003021F000270093730003C001E0009344
:100710007300032D003009F03A94042D003009F0E5
:100720004A94052D003009F05A9400E905BF9FBF97
:100730000F9178948895189518951895189518958F
:100740000F931F932F933F939FB724B135B100911F
:1007500071000236C9F1039500937100003249F12E
:10076000013469F100917200013069F00230B1F09A
:100770000091600010916100020F131F0093600050
:100780001093610021C00091620010916300020F7C
:10079000131F009362001093630016C00091640061
:1007A00010916500020F131F009364001093650001
:1007B0000BC001E00093720001E007B905C002E040
:1007C0000093720007E007B99FBF3F912F911F91DF
:1007D0000F911895F8940027009371000093720010
:1007E0000093600000936100009362000093630037
:1007F000009364000093650007B9789408951895F4
:0808000018951895189518953C
:00000001FF
